:100000000C948E000C94C7150C94AD000C94AD00AC
:100010000C94AD000C94AD000C94AD000C94320F18
:100020000C94AD000C94AD000C94AD000C94AD009C
:100030000C94AD000C94AD000C94AD000C94AD008C
:100040000C94AD000C94AD000C94AD000C94AD007C
:100050000C94AD000C94AD000C94AD000C94AD006C
:100060000C94AD000C94AD000C94AD000C94AD005C
:100070000C94AD000C94AD000C94AD000C94AD004C
:100080000C94AD000C94AD000C94AD00160C4E0C0D
:10009000680C680C960CA00CE30C3C0C910D100C39
:1000A000E80CED0CF30C0B0D0F0D240DBC0C290D01
:1000B000620D650D910D680D740D7B0D7E0D810D2A
:1000C000840D8B0D4C0D040309041C0348006500CE
:1000D0006E006E0069006E0067002000420065003F
:1000E0006B0065006C0012034B00650079006D0029
:1000F00061006E003600340012011001FF0000089C
:10010000501DE96000010102000109021200010115
:1001100000C03209040000000000000011241FBECE
:10012000CFEFD0E4DEBFCDBF18E0A0E0B1E0E4E067
:10013000F4E300E00BBF02C007900D92AE3DB107A3
:10014000D9F71AE0AEEDB8E001C01D92A337B107B0
:10015000E1F70E9406130C94001A0C940000EF9231
:10016000FF920F931F93CF93DF93EC017A018B01E2
:10017000B90120E030E040E050E016C0EA85FB85A0
:10018000E40FF51F80819181A281B3814C5F5F4FA5
:100190008E159F05A007B10729F4FB013183208349
:1001A00081E008C02F5F3F4F8C819D812817390760
:1001B00028F380E0DF91CF911F910F91FF90EF9096
:1001C0000895DC0120E030E01BC01696ED91FC9113
:1001D0001797A901440F551FE40FF51F0190F081F7
:1001E000E02D8181681751F41696ED91FC911797D7
:1001F000E40FF51F0190F081E02D0AC02F5F3F4F03
:100200008D919C91119728173907F8F2E0E0F0E002
:10021000CF0108950E94E10020E0892B09F421E03C
:10022000822F0895FC018485958520E0892B09F0B3
:1002300021E0822F0895FC01758764872485358528
:10024000C9010895DC0120E030E010C01696ED9160
:10025000FC911797C901880F991FE80FF91F0190AA
:10026000F081E02D838184832F5F3F4F8D919C919E
:1002700011972817390750F30895FC0161830895F9
:10028000FC01838184830895F8942CE088E190E058
:100290000FB6F894A895809360000FBE209360007D
:1002A000FFCF81E080933C0910923D0910923E09F6
:1002B00010923F09109240091092410908950E943E
:1002C00051018091740680937300E8E6F0E080812C
:1002D000886080837894089588E10FB6F8948093BD
:1002E0006000109260000FBE8FEF81B980EC82B980
:1002F00089E88AB980EF8BB90E945F01089581E097
:1003000080933C0910923D09089580E090E0FC0143
:10031000EE0FFF1FEE0FFF1FEE57F64F11821082F8
:1003200001968031910599F70895FF920F931F93DD
:10033000CF93DF93082F162FF42E882339F0C7E2CE
:10034000D0E048E250E066E270E006C0C4E2D0E0EF
:1003500045E250E063E270E020E030E0A12FB0E041
:10036000E22FCD01022E02C0959587950A94E2F7FF
:1003700080FD06C02F5F3F4F2830310589F7E0E050
:10038000F0E0802F90E0B3E0880F991FBA95E1F775
:10039000E82BF92BEE0FFF1FEE0FFF1FEE57F64F66
:1003A000718360831283F3828881912F90958923D2
:1003B0008883FA018081812B8083DF91CF911F9107
:1003C0000F91FF90089580E090E0FC01ED5FF54F04
:1003D0008083019680349105C1F708952091F1083A
:1003E0003091F208E091EF08F091F008E20FF31F6E
:1003F00080812F5F3F4F3093F2082093F10890E007
:10040000089585B7806885BF85B7806885BF0895E2
:100410008BB190917006892B8BB98BB190959823F5
:100420009BB908958BB190916E06892B8BB98AE1A7
:100430008A95F1F78BB1909598239BB908958BB16C
:1004400090916E06892B8BB9E8ECF0E03197F1F7CB
:100450008BB1909598239BB90895CF92DF92EF923C
:10046000FF920F931F93CF93DF938BB19091700600
:10047000892B8BB98BB1909598239BB9DD2400E033
:1004800010E0CC24C39423C089B190916F068923D6
:1004900039F4F701EE53F64FC082DD24D39406C041
:1004A000FE01E00FF11FEE53F64F1082E091E808D5
:1004B000F091E908099521960894E11CF11CC830D7
:1004C000D10511F7085F1F4F0034110521F07801A5
:1004D000C0E0D0E0D9CF8D2DDF91CF911F910F914A
:1004E000FF90EF90DF90CF90089592B12091710628
:1004F000822F8095892382B982B1822B82B9089597
:1005000082B190917106892B82B982B1909598231E
:1005100092B90895282FE82FF0E0EE5BF64F808126
:10052000882399F480917206662319F0922F982BF4
:1005300003C0982F9095922380917106982B92B9C1
:10054000E091E608F091E708099508951F938BB1B3
:1005500090917306892B8BB9E0EAFFE03197F1F7B0
:100560008BB1909598239BB910E0812F60E00E9499
:100570008A021F5F1034C9F71F9108951F939BB122
:1005800020917306822F809589238BB980EA9FE0A2
:100590000197F1F78BB1822B8BB910E0812F60E0CE
:1005A0000E948A021F5F1034C9F71F910895FF92BD
:1005B0000F931F93CF93DF93082FF62E142FC82F7E
:1005C000D0E0FE01EE5BF64F8081882319F0808138
:1005D0008417C1F4FE01EE5BF64F8081882321F47D
:1005E000802F6F2D0E948A02FF2009F410E0FE0187
:1005F000EE5BF64F10838081882321F4802F6F2DCE
:100600000E948A02DF91CF911F910F91FF90089570
:100610001F93CF93DF93C0E0D0E010E8DE01AE5728
:10062000B64F8D919C911197892BE1F0ED91FC9142
:100630001197808112969C911297892321F4139629
:100640008C9161E00CC01396EC911397F0E0EE5B97
:10065000F64F8081811731F413968C9160E0412F21
:100660000E94D70224961F5F1039C1F6DF91CF9107
:100670001F910895CF93DF93C0E0D0E0FE01ED5FBE
:10068000F54F8081FE01EE53F64F60810E948A0291
:100690002196C034D10591F7DF91CF910895DF9372
:1006A000CF930F92CDB7DEB78983898161E00E9435
:1006B0008A0288EC90E020E931E0F9013197F1F706
:1006C0000197D9F7898160E00E948A020F90CF914B
:1006D000DF910895DF93CF930F92CDB7DEB7898373
:1006E0008981E2ECF9E0E80FF11D80810F90CF9154
:1006F000DF910895DF93CF930F92CDB7DEB7898353
:100700008981E2ECF9E0E80FF11D808191E0892711
:100710000F90CF91DF910895DF93CF930F92CDB7D4
:10072000DEB78983898190E0803408F491E0892FD5
:100730000F90CF91DF910895DF93CF930F92CDB7B4
:10074000DEB789838981803440F50E942D02882399
:1007500021F1E981F0E0EE53F64F80818823E9F042
:1007600088EC90E020E931E0F9013197F1F7019749
:10077000D9F70E942D02882319F480E090E00EC082
:10078000E981F0E0EE53F64F808190E0882309F490
:1007900091E081E09827892F01C080E00F90CF91F0
:1007A000DF910895DF93CF930F92CDB7DEB78983A2
:1007B00089818034E0F40E942D02E981F0E0EE535B
:1007C000F64F8081882399F488EC90E020E931E0AD
:1007D000F9013197F1F70197D9F70E942D02E981CC
:1007E000F0E0EE53F64FE08181E0E82701C0E0E061
:1007F0008E2F0F90CF91DF9108950F931F9388EC68
:1008000090E020E931E0F9013197F1F70197D9F74C
:1008100089E361E00E948A0200EA1FE0C8010197B3
:10082000F1F788E00E944F0389E360E00E948A02AA
:10083000C8010197F1F71F910F9108950E94FD03E0
:100840000E94FD030895CF93DF93282FDB01EA0177
:1008500011961C921E928230A0F4882319F088E22F
:1008600090E002C085E290E011969C938E93222343
:1008700019F087E290E002C084E290E099838883D7
:1008800019C0E091430AF091440A84859585892B2B
:1008900089F00484F585E02D22508481281750F4D6
:1008A00085819681820F911D11969C938E93379628
:1008B000F983E88320E08D919C91892B09F021E058
:1008C000822FDF91CF910895CF93DF93DC01EB016D
:1008D00020E090E8FA0180818923ED91FC91119745
:1008E000882329F08881892339F480E306C0888130
:1008F000892311F488E701C081E3E20FF11D8083B1
:100900009695273011F02F5FE5CF8C9111969C9131
:10091000DF91CF910895CF92DF92EF92FF920F93E4
:100920001F93DF93CF9300D000D00F92CDB7DEB7E7
:100930008C01E091430AF091440A84859585892BC6
:1009400039F190E083E0C82ED12CCC0EDD1E7E0163
:100950000894E11CF11C12C0892F8E5FB701A6011B
:100960009D830E9423049D81882339F0E981FA81C7
:100970008081F801E90FF11D84839F5FE091430AB4
:10098000F091440A0484F585E02D8481981720F3C2
:1009900084B1F801808385B1818387B1828388B176
:1009A00083830F900F900F900F900F90CF91DF9156
:1009B0001F910F91FF90EF90DF90CF9008950F93CC
:1009C0001F930E942D0220E030E0022FF901EE5328
:1009D000F64F8081882339F0122F812F0E94D20395
:1009E0008823D9F306C02F5F3F4F2034310569F7C4
:1009F0000FEF802F1F910F910895FC0160E020817F
:100A00003181428153818091680390916903A09163
:100A10006A03B0916B03281739074A075B0709F48B
:100A200061E0862F0895FC0180916803909169032D
:100A3000A0916A03B0916B0380839183A283B383F7
:100A40001682EA5BFF4F1182108208950895282FC5
:100A500086958695869529F0A7E2B0E0E8E2F0E079
:100A600004C0A4E2B0E0E5E2F0E0277081E090E0AD
:100A7000382F01C0330F2A95EAF7232F662319F088
:100A80008081832B04C08081932F9095892380835C
:100A90008C91822B8C9308950F931F938C01FC01F2
:100AA000838161E00E942705F801808161E00E9456
:100AB0002705F801828161E00E9427051F910F91AF
:100AC0000895E091430AF091440A84859585892B25
:100AD00021F0848595850E944C050895FC01838151
:100AE00060E00E94270508950F931F938C01FC017D
:100AF000808160E00E942705F801808161E00E940A
:100B000027051F910F9108950F931F938C01FC01EE
:100B1000828160E00E942705F801828161E00E94E5
:100B200027051F910F910895FC0181810E942705DF
:100B30000895CF92DF92EF92FF920F931F93CF937E
:100B4000DF937C01DC0114968C91C82FD0E01EC08D
:100B5000D7011596ED91FC911697EC0FFD1FC08003
:100B600090E8D92E00E010E060E08D2D8C2109F096
:100B700061E0F70181810E942705C7010E94740589
:100B8000D6940F5F1F4F0830110571F72197FFEFC3
:100B9000CF3FDF07E9F6C7010E948405C7010E9425
:100BA0006E05DF91CF911F910F91FF90EF90DF9035
:100BB000CF900895CF92DF92EF92FF920F931F9301
:100BC000DF93CF9300D000D00F92CDB7DEB78C016A
:100BD000E091430AF091440A84859585892B79F147
:100BE00090E023E0C22ED12CCC0EDD1E7E010894B5
:100BF000E11CF11C13C0892F8E5FB701A6019D83F4
:100C00000E9423049D81882341F0E981FA81D80163
:100C1000A90FB11D14968C9180839F5FA091430A08
:100C2000B091440A1C96ED91FC911D978481981710
:100C300010F31C968D919C911D970E949905F801C7
:100C4000808184B9818185B9828187B9838188B99E
:100C50000F900F900F900F900F90CF91DF911F91F9
:100C60000F91FF90EF90DF90CF9008950F931F9317
:100C70008C01FC01858196810E94A417C8010E9405
:100C8000A4171F910F9108950E94A41708950F9320
:100C90001F938C01FC01848195810E94A417C801D7
:100CA0000E94A4171F910F9108950E94A417089500
:100CB0000F931F93CF93DF938C01C0E0D0E00AC065
:100CC000CE01880F991FE80FF91F808191810E9442
:100CD000A4172196D8018C9190E01596ED91FC9186
:100CE0001697C817D90764F3CF010E94A417C8014B
:100CF0000E94A417DF91CF911F910F9108950F9338
:100D00001F93CF93DF938C01C0E0D0E00AC0CE01E7
:100D1000880F991FE80FF91F808191810E94580662
:100D20002196D8018D919C9111971696ED91FC9189
:100D30001797C817D90758F3CF010E94A417C0E02E
:100D4000D0E00AC0CE01880F991FE80FF91F8081FB
:100D500091810E94A4172196F801828193810084D9
:100D6000F185E02DC817D90768F3CF010E94A417B9
:100D7000D8011A968D919C911B970E94A417C801C7
:100D80000E94A417DF91CF911F910F910895209198
:100D90006C0330916D03FC01EA5BFF4F6081718150
:100DA000C9018A5B9F4F0E94FA19089560916603FA
:100DB00070916703E091F608F091F708EA5BFF4F46
:100DC0007183608380916C0390916D038A5B9F4F68
:100DD0000E94FA19F8942CE088E190E00FB6F8949C
:100DE000A895809360000FBE20936000FFCF6091B4
:100DF0006C0370916D036A5F7F4F069640E450E08C
:100E00000E94CC190895EF92FF920F931F93CF93F6
:100E1000DF937C01C0916C03D0916D03DC011496CB
:100E2000ED91FC911597CE01049660810E94DC192A
:100E30008E010A5F1F4FD7011496ED91FC91159713
:100E40002596CE0161810E94DC192296D701149665
:100E5000ED91FC911597C80162810E94DC19D701C0
:100E60001496ED91FC911597CE01279763810E940E
:100E7000DC19E091430AF091440A84859585892B19
:100E8000D1F0289600E00DC0CE012196D70114962E
:100E9000ED91FC911597E00FF11D64810E94DC1922
:100EA0000F5FE091430AF091440A0484F585E02D38
:100EB0008481081748F3DF91CF911F910F91FF9024
:100EC000EF900895E091F608F091F70884819581FC
:100ED0000E948B048091F6089091F7080E94030706
:100EE0000895682F8091E0089091E1080196909311
:100EF000E1088093E00801970E94DC1980E090E00F
:100F00000895409168035091690360916A0370915C
:100F10006B0380916C0390916D030E94EE1908950C
:100F20000F931F938C014091680350916903609166
:100F30006A0370916B0380916C0390916D030E9422
:100F4000EE19C8010E94030760916C0370916D0354
:100F50006A5F7F4FC801069640E450E00E94CC19BA
:100F600080916C0390916D030A5B1F4FF8016081C3
:100F700071818A5B9F4F0E94FA191F910F9108950A
:100F800060916C0370916D036A5F7F4F069640E439
:100F900050E00E94AE190895CF92DF92EF92FF9237
:100FA0000F931F93CF93DF93C0916C03D0916D0388
:100FB000DC011496ED90FC901597CE0104960E94EA
:100FC000BE19F70180838E010A5F1F4F2596CE015F
:100FD0000E94BE19D70111968C932296C8010E94D7
:100FE000BE19F7018283CE0127970E94BE19D7014F
:100FF00013968C93C090430AD090440AF6018485DE
:101000009585892BA1F0289600E009C0CE01219694
:101010000E94BE19F701E00FF11D84830F5FD60116
:101020001C96ED91FC911D978481081778F3DF9150
:10103000CF911F910F91FF90EF90DF90CF90089587
:101040008091F6089091F7080E94CC07E091F6088D
:10105000F091F708848195810E94DA0508958091C6
:10106000E2089091E30801969093E3088093E208E8
:1010700001970E94BE1990E008950F931F938C0171
:1010800080916C0390916D030E94C619F8016083F2
:101090007183828393831F910F910895CF93DF9380
:1010A000EC0180916C0390916D030E94C6196883D6
:1010B00079838A839B8320916803309169034091EF
:1010C0006A0350916B03621773078407950781F4D5
:1010D000CE010E94CC0760916C0370916D036A5F32
:1010E0007F4FCE01069640E450E00E94AE190EC03C
:1010F000288339834A835B831E82CA5BDF4F198250
:101100001882C654D040CE010E949007DF91CF9143
:1011100008950F931F938C01862FF801648390E04C
:1011200061E070E00E94DB16F801858396831F91D1
:101130000F91089581E090E068E070E00E94DB1676
:10114000FC0114821682158210821182128213828F
:10115000089581E090E06CE170E00E94DB16089554
:10116000FF920F931F9381E090E068E470E00E948B
:10117000DB16F92E082F192F81E090E06CE170E06A
:101180000E94DB16F80184839583802F9F2D1F9189
:101190000F91FF90089581E090E065E070E00E947B
:1011A000DB16FC0188E0808311828FEF82838383CA
:1011B00014828E2F0895FF920F931F9381E090E089
:1011C00067E070E00E94DB16F92E082F192F81E0EE
:1011D00090E062E070E00E94DB16F8018583968360
:1011E00080915A03818380E4828381E083838483B6
:1011F000802F9F2D1F910F91FF900895FF920F93C5
:101200001F9381E090E06EE070E00E94DB16F92E03
:10121000082F192F81E090E062E070E00E94DB1659
:10122000F8018683978311861086138612861586A9
:101230001486118210821382128215821482802FEA
:101240009F2D1F910F91FF9008950E94DF048F3F03
:1012500051F1E5E9F8E001900020E9F73197E5590F
:10126000F840EF3319F410929508E0E0F0E0A5E9BA
:10127000B8E0EA0FFB1F80831182FD01019000207E
:10128000E9F73197EA1BFB0B6E2F4091F60850915E
:10129000F708742FFA0109C09D918681319698173D
:1012A00021F01092950820E014C08E2F871B86171E
:1012B00098F3FA013696DF010D900020E9F71197B7
:1012C000AE1BBF0B20E0862F90E08A179B0709F426
:1012D00021E0822F0895FC0181818430C9F185309D
:1012E00038F48230E9F1833068F4882359F04CC037
:1012F000863009F44BC0863008F441C0873009F0CD
:1013000043C02AC08093EA08868197819093EE08B3
:101310008093ED08828193819093F4088093F30881
:101320001092EC081092EB088091EF089091F00871
:10133000892B61F46091ED087091EE0881E090E0F6
:101340000E94DB168093EF089093F0088FEF0895CA
:1013500081E080933B0918C081E08093380914C074
:10136000E8EFF8E0F093540AE093530A019000206C
:10137000E9F73197E85FF8408E2F8F5F08958281FB
:1013800061E042E00E94D70280E00895828160E03F
:1013900042E00E94D70280E008954F925F926F92E0
:1013A0007F928F929F92AF92BF92CF92DF92EF92F5
:1013B000FF920F931F93CF93DF934C01DC010D90AD
:1013C0000020E9F76D010894C108D108C81AD90AAC
:1013D000AA24BB2403E070E9472E71E0572E60EA8F
:1013E000662E6FE0762E48C0F401EA0DFB1D808169
:1013F000809F70011124EEE6F3E0EE0EFF1EC0E0C8
:10140000D0E031C0D701ED91FC91EC0FFD1F808140
:10141000282F30E0207C30702038310519F48F738C
:1014200061E005C02034310541F48F7360E00E9413
:101430008A02C3010197F1F715C0203C310591F4F0
:10144000182F1F738091DF08181739F488EC90E08B
:10145000F2013197F1F70197D9F7812F0E944F03DD
:101460001093DF082196F701828190E0C817D90711
:1014700048F20894A11CB11CAC14BD0408F4B4CF0C
:10148000DF91CF911F910F91FF90EF90DF90CF9060
:10149000BF90AF909F908F907F906F905F904F9094
:1014A0000895CF93DF93EB0118820E94CD090E942B
:1014B000DF048F3FE1F3FE0101900020E9F731974F
:1014C000EC1BEF3311F41882E0E09E012E0F311D6A
:1014D000F90180831182883029F40E94FD03DF9195
:1014E000CF91089580E091E0E0CF4091ED085091D8
:1014F000EE088091EF089091F00861E070E026E737
:1015000036E00E9451192091ED083091EE0840E03C
:101510008217930709F441E0409338090895CF9268
:10152000DF92EF92FF920F931F93CF93DF938C0183
:101530007B016A01C0E0D0E017C0D8011896ED9198
:10154000FC911997CE01880F991FE80FF91F808130
:101550009181B7010E94F018009729F4F601D18318
:10156000C08381E00AC02196D80112968D919C918A
:101570001397C817D90708F380E0DF91CF911F9127
:101580000F91FF90EF90DF90CF900895CF92DF9270
:10159000EF92FF920F931F93DF93CF93CDB7DEB7F8
:1015A000C058D0400FB6F894DEBF0FBECDBF198231
:1015B0001A821B821C828CE3FE013596DF01982F74
:1015C0001D929A95E9F7B1E4CB2ED12CCC0EDD1EFD
:1015D000D6011D921D921D921C921397FE01EB5B8A
:1015E000FF4FDF011D928A95E9F782E091E07E01CD
:1015F0000894E11CF11CB7010E94510A87E191E0B7
:10160000B6010E94510AF70101900020E9F78F010D
:10161000015010400E191F09F60101900020E9F752
:101620003197EC19FD090E171F07F1F5C701B60137
:101630000E94F0180097C1F50130110549F4898125
:10164000883031F4E091F608F091F70816820CC06A
:101650008091F6089091F7080696BE016F5F7F4F64
:1016600040E450E00E9400198091F6089091F7083C
:1016700060916C0370916D036A5F7F4F069640E442
:1016800050E00E94CC198DE291E00E94CD09E091DA
:10169000F608F091F7088681882319F08BE391E032
:1016A00005C08FE391E002C087E491E00E94CD097C
:1016B0000E941E04C058DF4F0FB6F894DEBF0FBE65
:1016C000CDBFCF91DF911F910F91FF90EF90DF90F1
:1016D000CF9008959F92AF92BF92CF92DF92EF92F8
:1016E000FF920F931F93DF93CF9300D00F92CDB74C
:1016F000DEB78BE090E061E070E00E94DB168C01C9
:1017000069E671E00E94F9180E5F1F4F1B830A8380
:10171000025010408FEF898382E0C82ED12CCC0E6E
:10172000DD1EC60165E270E044E250E00E94640400
:10173000C8010E94CD09C60168E270E047E250E0AE
:101740000E946404F80180818F5F8083C8010E9439
:10175000CD09E091430AF091440A84859585892B4F
:1017600009F1A484B584FF24C6019C2CE92E6E01E6
:101770000894C11CD11C12C0F501658176816F0DE2
:10178000711D892D9E2DA6010E946404F80180819F
:101790008F5F8083C8010E94CD09F394F501848195
:1017A000F81650F30E94FD03C8010E94A4170F9081
:1017B0000F900F90CF91DF911F910F91FF90EF90BD
:1017C000DF90CF90BF90AF909F900895EF92FF92DF
:1017D0000F931F93DF93CF9300D000D0CDB7DEB728
:1017E0007C018B01DB0111968C91BE016F5F7F4FF5
:1017F000AE014D5F5F4F0E942304882309F4A2C10C
:10180000F8018081E82FF0E0ED31F10508F089C1A1
:10181000EA5BFF4FEE0FFF1F0590F491E02D099456
:10182000D80113968C918093020A7BC1F801428102
:10183000242F90E002C026959F5F20FFFCCFD801A7
:1018400013968C911397282330E002C0220F331F88
:101850009A95E2F7E981FA81808140954823408397
:10186000E981FA818081822B8083EB81FC818081F8
:1018700012969C91892B10C0EB81FC818081D8014C
:1018800012969C911297892B8083E981FA8190812D
:1018900012968C9180958923808343C1E981FA81D6
:1018A0009081F80132819323EB81FC818081832B2D
:1018B0008083E981FA812081D80112968C918095EC
:1018C00082238083E981FA8180819327982BBAC093
:1018D000F8014281E981FA812081823011F03FEFE5
:1018E00001C031E02423842F90E003C08695269523
:1018F0009F5F80FFFBCF230F282330E002C0220F21
:10190000331F9A95E2F7EB81FC818081842B8083E1
:10191000E981FA819081D80112968C918095892372
:101920008083E981FA818081822BB6CFEB81FC81B3
:101930009081D80112968C91129780958923A4CF1B
:10194000F801938180E0228130E0822B932B9C016F
:10195000442737FD4095542F60EA7FE007C0CB0154
:101960000197F1F72150304040405040211531059A
:1019700041055105A1F7D5C0D7011A96ED91FC910B
:101980001B97D80113969C91139780E012962C9187
:1019900030E0822B932B880F991F880F991FE80F37
:1019A000F91F80819181A281B38120EA3FE006C0C6
:1019B000F9013197F1F70197A109B1090097A10544
:1019C000B105B1F7AEC0F80183810E94F90DA9C03D
:1019D000D80113968C9161E003C0F801838160E027
:1019E0000E948A029EC0D7011896ED91FC9119972A
:1019F000D80113969C91139780E012962C9130E0B9
:101A0000822B932B880F991FE80FF91F80819181FA
:101A10000E94CD0986C081E080933B0982C0F80115
:101A2000A281B0E0AD5FB54F9C918381E82FF0E0DB
:101A3000ED5FF54F80818C93D8011396EC91F0E027
:101A4000ED5FF54F90836DC0F80183810E944F03D5
:101A500068C0D80113968C91882361F48EEB92E0D4
:101A60009093E5088093E40885E792E09093E70877
:101A70008093E608F8018381813009F052C086EA3C
:101A800092E09093E5088093E40880E892E09093D8
:101A9000E7088093E60845C0D80113968C91882307
:101AA00031F48FE192E09093E9088093E808F8011F
:101AB00083818130B1F582E192E09093E9088093CF
:101AC000E8082FC00E9462072CC00E94200829C08D
:101AD000D80111968C91119712966C9112971396CA
:101AE0004C910E9495011DC088EF98E00E94CD099D
:101AF0000E941E0416C00E946A0B13C00E94250E8D
:101B000010C00E94C60A0DC08091390990913A090F
:101B10000E948B0406C08091390990913A090E9475
:101B2000DA05E091430AF091440A84859585892B72
:101B300049F0D80111968C91823020F084859585EA
:101B40000E9499050F900F900F900F90CF91DF9109
:101B50001F910F91FF90EF9008950F931F93CF93D4
:101B6000DF93EC0100E010E021C0C801880F991F4D
:101B7000ED81FE81E80FF91F0190F081E02D848155
:101B8000882359F0803421F48A81803469F405C0B7
:101B9000803651F48A81803639F48091430A9091DD
:101BA000440ABF010E94E60B0F5F1F4F888190E03F
:101BB00008171907D4F28A81803411F080E401C03B
:101BC00080E68A83DF91CF911F910F910895CF9383
:101BD000DF93EC018C81882349F081508C8388232A
:101BE00029F4CE010E94AD0D8B818C83DF91CF91C2
:101BF00008951F93CF93DF93182FC0E0D0E012C059
:101C00000680F781E02DCE01880F991FE80FF91F9C
:101C10000190F081E02D8181181719F4CF010E9405
:101C2000AD0D2196E091430AF091440A80819181A3
:101C3000C817D90728F3DF91CF911F91089589EF35
:101C40000E94F90D1092DE080895E091F608F091D7
:101C5000F7088681882339F08AEF0E94F90D82E027
:101C60008093DE08089585E791E00E94CD090E94E7
:101C70001E0408958F929F92AF92BF92CF92DF92EF
:101C8000EF92FF920F931F93CF93DF938C015B0131
:101C9000CC24DD24E0EA8E2EEFE09E2E48C0D80151
:101CA0001696ED91FC9117977601EE0CFF1CEE0D48
:101CB000FF1D0190F081E02D918180915A039817CA
:101CC00099F5C0E0D0E021C0D8011696ED91FC91C5
:101CD0001797EE0DFF1D0190F081E02DCE01880FCA
:101CE000991F0580F681E02DE80FF91F6081718151
:101CF000C8010E94E60BA114B10431F0C501F40142
:101D00003197F1F70197D9F72196D8011696ED9101
:101D1000FC911797EE0DFF1D0190F081E02D808161
:101D200090E0C817D90784F20894C11CD11CF801AF
:101D300080819181C816D90608F4B1CFDF91CF9187
:101D40001F910F91FF90EF90DF90CF90BF90AF90D9
:101D50009F908F900895DF93CF9300D0CDB7DEB7DB
:101D600019821A8280913E09843031F1853040F425
:101D7000823099F08330A8F4813009F06EC008C039
:101D80008630B1F18630E8F0873009F066C05EC079
:101D900080913F090E94F90D60C080913F0961E088
:101DA00003C080913F0960E041E00E94D70280EAD1
:101DB0009FE00197F1F751C080913F090E944F03C6
:101DC0004CC0809140092091400940913F0990E02A
:101DD000F3E096958795FA95E1F7277061E070E05A
:101DE00002C0660F771F2A95E2F781700E94950165
:101DF0000E94CB08FC0180914009869586958695C6
:101E0000818320914009277081E090E002C0880F13
:101E1000991F2A95E2F7828380913F09838381305D
:101E200039F0813018F0823039F404C087E005C001
:101E3000108204C084E001C088E080838091430A5E
:101E40009091440ABF010E94E60B07C080913F09B0
:101E50008983CE0101960E94CD090F900F90CF91FA
:101E6000DF9108951F920F920FB60F920BB60F924B
:101E700011242F933F934F935F936F937F938F938F
:101E80009F93AF93BF93EF93FF9389B190917406A3
:101E9000892309F041C089B190917506892339F0F1
:101EA00090913D0980913C09892B80933D09809157
:101EB0003C09880F80933C0980913C09882361F597
:101EC00080914109882369F480913D0980933E09FE
:101ED000E0913E09F0E0E25AFC4F80818093410995
:101EE0000DC080914109815080934109E0914109E1
:101EF000F0E080913D09E45CF64F838380914109D5
:101F0000882329F40E94AB0E0E94510105C081E094
:101F100080933C0910923D09FF91EF91BF91AF91E1
:101F20009F918F917F916F915F914F913F912F91F1
:101F30000F900BBE0F900FBE0F901F901895EF9251
:101F4000FF920F931F93CF93DF9380E090E0FC010B
:101F5000E850F74F1082019680349105C1F7C8E828
:101F6000D1E0EE24FF2481E08F1530F488818032A7
:101F700019F48981803259F00E2D10E0898190E0AA
:101F80000E94D8180850174FF8018083E394F39407
:101F90002196F1E2FF1639F7DF91CF911F910F9152
:101FA000FF90EF900895F8940E949D14519A88E84C
:101FB00093E120E931E0F9013197F1F70197D9F781
:101FC000519878941092F0081092EF080895EF92CB
:101FD000FF920F931F938C017B01CB010E940F197D
:101FE000F801848390E061E070E00E94DB16F80164
:101FF00085839683C7010E940F19F8018083C7016A
:102000000E940F19F8018183C7010E940F19F8017E
:102010008283C7010E940F19F80183831F910F91DA
:10202000FF90EF900895EF92FF920F931F937C0122
:102030008B01CB010E940F19F7018083C8010E9418
:102040000F19F7018483C8010E940F19F7018183DA
:10205000C8010E940F19F7018283C8010E940F195D
:10206000F70183831F910F91FF90EF900895EF92F6
:10207000FF920F931F938C01F62EE72EDC016C91DB
:1020800070E06F5F7F4F660F771F15968D919C9163
:1020900016970E94FC17F80196838583E081F0E093
:1020A000EE0FFF1FE80FF91FF082E182D8018C913B
:1020B0008F5F8C938F2D9E2D1F910F91FF90EF902E
:1020C0000895CF92DF92EF92FF920F931F93CF93D9
:1020D000DF936C018B01CB010E940F19F601838302
:1020E000C8010E940F19C0E0D0E0E82EFF240AC00A
:1020F0000E94CB08BC01C6010E943710B8010E94A3
:1021000013102196CE15DF059CF3DF91CF911F911F
:102110000F91FF90EF90DF90CF900895EF92FF9294
:102120000F931F938C01F62EE72EDC0116968D91EE
:102130009C9117976D917C916F5F7F4F660F771F12
:102140000E94FC17F801978386830680F781E02DB3
:10215000D8018D919C911197880F991FE80FF91F55
:10216000F082E1828D919C911197019611969C933A
:102170008E938F2D9E2D1F910F91FF90EF900895BC
:10218000FF920F931F93CF93DF938C01F62E0E9443
:102190000A01882331F4C8016F2D0E94E100EC018F
:1021A00008C00E94DB08EC01F982C801BE010E9450
:1021B0008E10CE01DF91CF911F910F91FF90089566
:1021C000CF92DF92EF92FF920F931F938C016A01DF
:1021D0007B01DC011A968D919C911B9714966D9151
:1021E0007C9115976F5F7F4F660F771F660F771F84
:1021F0000E94FC17F801938782870284F385E02D03
:10220000D80114968D919C911597880F991F880F6E
:10221000991FE80FF91FC082D182E282F3821496DF
:102220008D919C911597019615969C938E9314977A
:1022300014962D913C91159721503040C9011F9162
:102240000F91FF90EF90DF90CF900895AF92BF92E3
:10225000CF92DF92EF92FF920F931F937C01B62EE5
:10226000A72EFC0180859185628173816F5F7F4F0E
:10227000660F771F0E94FC17F70191878087C08443
:10228000D18402811381EB2DFA2DDF010D90002006
:10229000E9F7CD018E1B9F0B61E070E00E94DB1619
:1022A000000F111F0C0D1D1DF80180839183F70194
:1022B0002085318582819381EB2DFA2DDF010D90F0
:1022C0000020E9F71197AE1BBF0B880F991F280F4D
:1022D000391FF901808191816B2D7A2DAD010E940A
:1022E0000019F70182819381019693838283228171
:1022F000338121503040C9011F910F91FF90EF9021
:10230000DF90CF90BF90AF9008959F92AF92BF9211
:10231000CF92DF92EF92FF920F931F93CF93DF93B1
:102320005C016BEA71E00E942611C50164EA72E06B
:102330000E942611C50168E473E00E9426110E94E4
:10234000DB088C0182E3F80181830E94CB08FC0149
:102350002CE0D22ED08212821382C801BF010E94CB
:102360003710C501B8010E948E100E94CB087C0175
:102370008DE0F70180830E94DB088C0183E2F80185
:102380008183C801B7010E943710C501B8010E94BE
:102390008E100E94DB088C018AE2F80181830E9482
:1023A000CB08FC01D08281E082831382C801BF0187
:1023B0000E943710C0E0D0E09FE0992E85E2C82E41
:1023C000B5E0FB2EA8EEDA2EF3E0EF2E0E94CB084C
:1023D000FC019082C382C801BF010E9437100E9495
:1023E000CB08FC01F082D282E382C801BF010E94C7
:1023F00037102196CA30D10549F70E94CB08FC015D
:102400008CE0808382E082831382C801BF010E9436
:102410003710C501B8010E948E100E94DB088C01A4
:102420008BE3F80181830E94CB08FC0186E1808365
:1024300012821382C801BF010E943710C501B80182
:102440000E948E1081E0DF91CF911F910F91FF903C
:10245000EF90DF90CF90BF90AF909F9008952F9214
:102460003F924F925F926F927F928F929F92AF9224
:10247000BF92CF92DF92EF92FF920F931F93DF9361
:10248000CF93CDB7DEB7C050D0410FB6F894DEBFC2
:102490000FBECDBF1C012B01CB010E940F19982F3D
:1024A00080915703981749F4C2010E940F19982F81
:1024B00080915803981709F485C0892F90E0B201E4
:1024C0000E94941980E088C080915B03181701F581
:1024D00000E010E009C0E1E0F0E0EC0FFD1FE00FCC
:1024E000F11F80830F5F1F4FC2010E940F198823C5
:1024F00091F781E090E08C0F9D1F080F191FF801E4
:102500001082C101BE016F5F7F4F0E9426115AC029
:1025100080915C031817E1F5C2010E940F193C017C
:10252000C2010E940F197C01C2010E940F195C01B7
:10253000C2010E940F190027F7FC0095102F102FE1
:102540000F2DFE2CEE24CC24B7FCC094DC2C6501AE
:10255000BB24AA24EA28FB280C291D29882477FCFF
:102560008094982CE628F72808291929AA2797FD8E
:10257000A095BA2FB82FAA2799278827E82AF92AE1
:102580000A2B1B2BC101B801A7010E94E0101AC041
:1025900080915D03181759F40E949A08F1019587FC
:1025A000848784859585B2010E94E70F0BC00E9445
:1025B000DB08BC01C1010E948E10FC011183B20135
:1025C0000E946110C2010E940F19182F80915903B7
:1025D000181709F079CF81E0C050D04F0FB6F894AA
:1025E000DEBF0FBECDBFCF91DF911F910F91FF9046
:1025F000EF90DF90CF90BF90AF909F908F907F90A3
:102600006F905F904F903F902F900895CF92DF9200
:10261000EF92FF920F931F93CF93DF930E946C0171
:1026200080E090E0FC01ED5FF54F808301968034FF
:102630009105C1F780E090E0FC01EE0FFF1FEE0F67
:10264000FF1FEE57F64F11821082019680319105DF
:1026500099F70E949F0F8FE08093020A10923B0926
:102660001092380986EA92E09093E5088093E40896
:1026700080E892E09093E7088093E60882E192E098
:102680009093E9088093E8080E94FE088093430A2B
:102690009093440A66E776E00E942F12882331F473
:1026A0008091430A9091440A0E948511E091E408C8
:1026B000F091E50809950E942D020E943A030E94BC
:1026C00061050E94B0089093F7088093F6080E9475
:1026D0004E0881E090E06CE170E00E94DB16809390
:1026E000390990933A090E948B048091430A909192
:1026F000440A60E070E00E943A0E0E94D30FFF246B
:10270000F394E0E9CE2EE1E0DE2EEE24E3940E9485
:10271000A41480913B09882321F4809138098823EF
:10272000F1F084EC99E0F6013197F1F70197D9F7D0
:1027300080913B09882311F00E94D60680913809C8
:10274000882369F0F8942CE088E190E00FB6F894C3
:10275000A895809360000FBE20936000FFCF0E9479
:1027600008038091DE08813081F1813018F08230D9
:1027700071F661C08091020A0E949C03882311F1C6
:10278000A091430AB091440A20E030E010C01696B0
:10279000ED91FC911797C901880F991FE80FF91F58
:1027A0000190F081E02D838184832F5F3F4F8D91D5
:1027B0009C9111972817390750F3E092DE08FF2407
:1027C000F394A5CF0E943A03A2CF8091020A0E94FF
:1027D000D203882319F400E010E023C0FF2021F089
:1027E0008091020A0E944F031092DE0890CF06806B
:1027F000F781E02DC801880F991FE80FF91FC081EC
:10280000D18189810E949C03882349F0CE010E94D6
:10281000E70D89810E94D2038823D9F3FF240F5F3B
:102820001F4FE091430AF091440A8081918108177B
:102830001907E8F26CCF0E942509882309F467CFB5
:102840000E941F0E64CF0F931F930E94FE08182F43
:10285000092F1092F2081092F10864E876E00E94C5
:102860002F12882341F06091F3087091F408812FB2
:10287000902F0E943A0E812F902F0E947F061F9169
:102880000F9108950F931F93CF93DF938C01C09105
:10289000EF08D091F00840E050E070E016C0E09101
:1028A000EB08F091EC08EC0FFD1FD801A40FB51F49
:1028B0008C9180834F5F5F4F8091EB089091EC0883
:1028C00001969093EC088093EB082091EB083091EF
:1028D000EC088091ED089091EE082817390718F45C
:1028E00046175707E4F22091EB083091EC088091ED
:1028F000ED089091EE082817390710F480E018C011
:102900008091EA08882319F40E94231406C080915C
:10291000EA08833011F40E94750A8091EF089091C3
:10292000F0080E94A4171092F0081092EF0881E0BE
:10293000DF91CF911F910F910895E9E6F0E080813A
:1029400082608083E89A08951F93CF93DF9360910C
:10295000550A635067FDA6C08091520ACCE0D0E0D2
:10296000C81BD109C75AD54F8091510A8D3209F041
:1029700086C0683009F094C083EC8093450A8AE5EC
:102980008093D5081092F5089881892F807641F0C0
:10299000CE010E946B09282F8F3F09F45FC065C0EC
:1029A0002A8110924E0A8981882349F49F7119F473
:1029B00081E080934E0A10924F0A22E048C0853091
:1029C00019F42093560A42C0863089F58B818130F4
:1029D00019F488EF90E020C0823019F48AE091E089
:1029E0001BC08330F9F48A81882341F486EC90E09F
:1029F0009093540A8093530A24E015C0813041F427
:102A00008AEC90E09093540A8093530A2CE10BC017
:102A1000823041F486EE90E09093540A8093530AFA
:102A200022E101C020E080E48093F5081EC08830D8
:102A300021F421E088E59AE00CC0893019F4209354
:102A4000580A04C08A3011F421E001C020E08EE46D
:102A50009AE09093540A8093530A07C0888187FDB7
:102A60002E8180E88093F50806C08F81882319F4B1
:102A70008E81821708F0822F8093D60811C0809132
:102A8000F50887FF0DC0CE010E9442148F3F21F44C
:102A90008EE18093D50804C0882311F01092D608E7
:102AA0001092550A8091D50884FF4AC08091D608BB
:102AB0008F3F09F445C0182F893008F018E0811BBA
:102AC0008093D6088091450A98E889278093450A23
:102AD000112341F12091530A3091540A8091F50855
:102AE00086FF0DC0A6E4BAE080E090E0F901E80FAF
:102AF000F91FE491ED9301961817C1F708C0912FC3
:102B0000D901E6E4FAE08D9181939150E1F71150FB
:102B1000812F90E01F5F0196820F931F9093540ABC
:102B20008093530A86E49AE0612F0E94C315612FB7
:102B30006C5F6C3019F08FEF8093D6086093D508E6
:102B400094E189B1867031F49150D9F71092560A08
:102B50001092500ADF91CF911F910895A82FB92F9D
:102B600080E090E041E050EA609530E009C02D91AE
:102B700082279795879510F084279527305EC8F3B4
:102B80006F5FA8F30895EADF8D939D930895CF9327
:102B9000CFB7CF93DF93C395499BE9F7499B0BC010
:102BA000499B09C0499B07C0499B05C0499B03C07D
:102BB000499B01C089C06F93C091520ADD27C75A53
:102BC000D54F2F9365E5499B03C02F916F91E6CFB9
:102BD0000F931F934F9320E040E15F9309B106707C
:102BE00001FB27F93F9350E03BE039C01670406489
:102BF0002F77012F5F5F1EC0406819B116702F77C5
:102C000052501FC0406409B12F770670D1F15F5F49
:102C100000C023C0406219B12F77167091F15F5F39
:102C200000C025C006701027515012F45D5F0000EF
:102C3000115027952C3F19B1C8F616700127015085
:102C400027952C3FC8F64227499309B106701027F3
:102C50004F73115027952C3FA8F64695469519B10C
:102C6000167079F00127015027952C3F98F66B5A82
:102C700060F3315009B1B0F600C011E01CBB002771
:102C800017C03B503195C31BD04011E01CBB0881DD
:102C9000033CF9F00B34E9F02091500A1981110F2F
:102CA0001213EDCF093651F10D3211F0013E39F713
:102CB0000093570A3F915F914F911F910F912F9170
:102CC0006F91CCB3C0FD67CFDF91CF91CFBFCF91D4
:102CD00018952091570A222369F31091550A112360
:102CE00039F534303AF13093550A2093510A109156
:102CF000520A3BE0311B3093520A1CC00091550A26
:102D00000130B4F40AE53091D50834FD14C00093C5
:102D1000D508C5E4DAE013C0052710E000C00000C4
:102D20000BB91AC0052710E0221F1DC010E021C0FA
:102D30004AE502C032ED432FC4E1D0E032E01AB1DF
:102D40001660599A0BB11AB956E020E865E320FFE6
:102D500005270BB9279517951C3FF0F66695B8F730
:102D6000B1F720FF05270BB9279517951C3FD0F623
:102D70002795179517FF052700001C3F0BB9B0F6E4
:102D800029913A9519F7097F1091560A110FC651EA
:102D9000D0400BB911F01093500A11E01CBB026037
:102DA0001AB1197F402F497F54E05A95F1F70BB9BA
:102DB0001AB94BB97FCF0F931F93CF93DF93689FBF
:102DC0008001699F100D789F100D1124C8010E9489
:102DD000F716EC01009729F060E070E0A8010E946E
:102DE000E918CE01DF91CF911F910F910895CF93F4
:102DF000DF93BC018230910510F462E070E0A09195
:102E0000710AB091720AED01E0E0F0E040E050E0BC
:102E100021C0888199818617970769F48A819B81EF
:102E2000309719F09383828304C09093720A809341
:102E3000710AFE0134C06817790738F4411551054D
:102E400019F08417950708F4AC01FE018A819B8173
:102E50009C01E9012097E9F641155105A9F1CA0144
:102E6000861B970B049708F4BA01E0E0F0E02AC053
:102E70008D919C91119784179507F9F46417750744
:102E800081F412968D919C911397309719F093834A
:102E9000828304C09093720A8093710AFD01329676
:102EA0004FC0CA01861B970BFD01E80FF91F619304
:102EB000719302978D939C9343C0FD01828193810E
:102EC0009C01D9011097A1F680916F0A9091700A28
:102ED000892B41F48091D9089091DA089093700A77
:102EE00080936F0A4091DB085091DC084115510531
:102EF00041F44DB75EB78091D7089091D808481B30
:102F0000590B20916F0A3091700A24173507B0F4DD
:102F1000CA01821B930B8617970780F0AB014E5FA7
:102F20005F4F8417950750F0420F531F5093700A5C
:102F300040936F0AF9016193719302C0E0E0F0E001
:102F4000CF01DF91CF910895CF93DF93009709F4DC
:102F500050C0EC0122971B821A82A091710AB09195
:102F6000720A109709F140E050E0AC17BD0708F174
:102F7000BB83AA83FE0121913191E20FF31FAE17AB
:102F8000BF0779F48D919C911197280F391F2E5FFF
:102F90003F4F3983288312968D919C9113979B8381
:102FA0008A834115510571F4D093720AC093710A56
:102FB00020C012968D919C911397AD01009711F04E
:102FC000DC01D3CFFA01D383C28321913191E20F87
:102FD000F31FCE17DF0769F488819981280F391F05
:102FE0002E5F3F4FFA01318320838A819B81938337
:102FF0008283DF91CF9108958F929F92AF92BF927B
:10300000CF92DF92EF92FF920F931F93CF93DF93B4
:103010008C01009729F4CB010E94F7168C01BAC0ED
:103020009EEFE92E9FEFF92EE00EF11E5801A60E3D
:10303000B71EAE14BF0408F4ABC08EEF882E8FEF1E
:10304000982E8A0C9B1CE701488159814617570727
:10305000B8F04530510508F49DC0CA0104978617A1
:10306000970708F497C042505040461B570BF40195
:103070005183408379836883C5010E94A4178AC065
:103080006B01C41AD50AE091710AF091720AA0E0AE
:10309000B0E0C0E0D0E042C0E815F905A1F520811C
:1030A00031812C153D0578F1C90102968C159D05DD
:1030B000A8F04E5F5F4F420F531FE70159834883CB
:1030C00022813381109729F013963C932E93129707
:1030D00061C03093720A2093710A5CC02250304064
:1030E0002C193D0931832083109729F01396FC9306
:1030F000EE93129704C0F093720AE093710AF701FD
:103100007183608347C080819181C817D90708F413
:10311000EC01DF01828193819C01F901309709F074
:10312000BBCF400F511F80916F0A9091700A841796
:103130009507E9F4C617D707D0F42091DB08309142
:10314000DC082115310541F42DB73EB78091D70831
:103150009091D808281B390BA216B306C8F4B09278
:10316000700AA0926F0AE7017983688313C0CB01CC
:103170000E94F716EC01009759F0F7014081518148
:10318000B8010E94E018C8010E94A4178E0102C075
:1031900000E010E0C801DF91CF911F910F91FF90E7
:1031A000EF90DF90CF90BF90AF909F908F90089559
:1031B0009111089581548A5108F4805E855A0895CA
:1031C000FB01DC0102C001900D9241505040D8F744
:1031D0000895DC0101C06D9341505040E0F708951F
:1031E000FB01DC018D91019080190110D9F3990B3D
:1031F0000895FB01DC0101900D920020E1F7089594
:10320000FB01DC014150504048F001900D9200203C
:10321000C9F701C01D9241505040E0F70895CF9387
:10322000DF93EC014B8140FF1AC046FF0AC04F7B81
:103230004B838E819F8101969F838E838A81282F65
:103240002BC042FF13C0E881F9818081282F3327EA
:1032500027FD30952115310529F440624B832FEF6E
:103260003FEF1BC03196F983E88311C0EA85FB85E7
:10327000CE0109959C0197FF0AC09B812F5F3F4FAC
:1032800011F080E201C080E1892B8B83E8CF8E8131
:103290009F8101969F838E8330E0C901DF91CF919A
:1032A00008958F929F92AF92BF92CF92DF92EF924A
:1032B000FF920F931F93CF93DF93FC014B015A01B1
:1032C0006901D90113968C9181FF1EC07F01C0E076
:1032D000D0E014C0D6011896ED91FC911997D70152
:1032E0008C91B6010995892B89F40894E11CF11C95
:1032F0000F5F1F4F0815190568F32196CA15DB05E6
:1033000028F400E010E0F6CFC0E0D0E0CE01DF917D
:10331000CF911F910F91FF90EF90DF90CF90BF90D2
:10332000AF909F908F9008959C01FB01838180FF57
:1033300011C086FD0FC09FEF2F3F390759F0228340
:1033400080648F7D838386819781019797838683AD
:1033500030E002C02FEF3FEFC9010895DC01CB013F
:10336000FC01F999FECF06C0F2BDE1BDF89A319695
:1033700000B40D9241505040B8F70895F999FECF2E
:1033800092BD81BDF89A992780B50895A6E1B0E075
:1033900044E050E00C94B019DC01A40FB51F41507B
:1033A000504048F0CB01840F951F2E910E94DD19EB
:1033B00041505040D0F70895262FF999FECF92BD85
:1033C00081BDF89A019700B4021639F01FBA20BDEA
:1033D0000FB6F894FA9AF99A0FBE08950396272F1C
:1033E0000E94DD190E94DC19252F0E94DD19242F6F
:1033F0000C94DD190196272F0E94DD190C94DC191D
:04340000F894FFCF6E
:103404002A00656E746572206E657720706173732F
:10341400776F72643A2000726570656174206E651E
:10342400772070617373776F72643A20006F6B2C2E
:103434002070617373776F72642000736574006326
:103444006C65617265640070617373776F72647325
:10345400206469666665722C206E6F7468696E6795
:10346400206368616E6765640061203030303030FD
:103474003030300A006E6F2070617373776F72643E
:1034840020646566696E6564006669726D77617251
:103494006520312E36205365702031312032303191
:1034A400372030383A34323A3137000C0A202A2A8D
:1034B4002A2A2A206B65796D616E3634207665720E
:1034C40073696F6E20312E36207265616479202A0B
:1034D4002A2A2A2A0A0A202020206E6F20636F6E6F
:1034E40066696775726174696F6E20666F756E6464
:1034F40020696E20656570726F6D0A20202020207F
:10350400207573696E672066616C6C6261636B2001
:10351400636F6E66696775726174696F6E0A0A20FB
:103524002020202020205F763A2074797065206660
:1035340069726D776172652076657273696F6E0A60
:10354400202020202020205F623A20656E7465725E
:1035540020626F6F746C6F616465720A2020202092
:103564002020205F663A2074657374206372797337
:1035740074616C206672657175656E63790A2020CA
:1035840020202020205F743A2074797065207468AC
:103594006973206D6573736167650A0A7265616496
:1035A400792E0A000C0A202A2A2A2A2A20206B654E
:1035B400796D616E3634206672657175656E6379F6
:1035C400207465737420202A2A2A2A2A0A0A696622
:1035D4002074686520666F6C6C6F77696E67207401
:1035E400656E20646F747320617265206E6F742041
:1035F40074797065640A776974682061626F7574A0
:10360400206F6E65207365636F6E642064656C6102
:103614007920696E206265747765656E2C0A63682B
:1036240065636B2061746D656C20667573657320CA
:10363400616E642F6F72206372797374616C20639E
:103644006972637569740A000A0A72656164792E85
:103654000A0000406040601CCFFFFEFDFCFB00013F
:10366400010101020201B0B03412CDABB80FDF0882
:1036740000DF0800DF0800920601DF08009306035C
:10368400DF0800DF0800DF0800DF0800960603DF1C
:1036940008009906039C0601DF0800DF0800DF0824
:1036A400009D06019E0603A10601A20601DF080093
:1036B400DF0800DF0800DF0800DF0800DF0800DFA4
:1036C4000800A30603A60601A70603AA0603AD067F
:1036D40001AE0603B10603B40603B70603BA060334
:1036E400BD0603C00603C30603C60603C90601CA12
:1036F4000601CB0601CC0601CD0601CE0601CF069C
:1037040001D00601D10601D20601D30601D4060177
:10371400D50601D60601D70601D80601D90601DA75
:103724000601DB0603DE0601DF0603E20603E50607
:1037340001E60603E90603EC0603EF0603F20603BB
:10374400F50603F80603FB0603FE0603010703045C
:1037540007030707030A07030D07031007031307EB
:10376400031607031907031C07031F070322070394
:103774002507032807032B07032E07033107033408
:1037840007033707013807033B07013C07013D07DF
:1037940003400701410701420701430701440701B0
:1037A4004507014607014707014807014907014A40
:1037B40007014B07014C07014D07014E07014F0755
:1037C4000150070151070152070153070154070132
:1037D4005507015607015707015807015907015AB0
:1037E40007035D0703600703630703660703DF0836
:1037F40000690703DF0800DF0800DF08006C070129
:103804006D07016E07016F070170070373070376E5
:1038140007037907037C0703DF0800DF08007F073D
:10382400038207038507038807038B07018C0703BB
:103834008F07039207039507039807039B07039ECB
:103844000703A10703A40703A70703AA0703AD07F8
:1038540001AE0703B10703B40703B70703BA0703AD
:10386400BD0703C00703C30703C60703C90703CC87
:103874000703CF0703D20703D50703D80703DB07E2
:1038840003DE0703E10703E40703E70703EA07038B
:10389400ED0703F00703F30703F60703F90703FC37
:1038A4000703FF07030208030508030808030B08BE
:1038B400030E08010F080110080111080112080184
:1038C4001308011408011508011608011708011846
:1038D40008011908011A08011B08011C08011D0828
:1038E400011E08011F080120080121080122080106
:1038F40023080124080125080126080127080128B6
:1039040008032B08032E080331080334080337087F
:10391400013808033B08033E080341080344080335
:103924004708034A08034D08035008035308035685
:1039340008035908035C08035F0803620803650869
:10394400036808036B08036E080371080374080313
:103954007708037A08037D08038008038308038635
:1039640008038908038C08038F08039208030810CE
:103974000140808040200000000300000000710727
:103984002F08000000000001000000000000EE010C
:103994000000FF97DF57B9C879B9DE79C8F897C432
:1039A40057DEC097C157D097DA5797C357E7B9C7BF
:1039B40079B9DF79B9C179B9D979B9C279B9DA797B
:1039C400B9C379B9DB79B9C479CEC5FDDDE5FEDCCF
:1039D400C7DFC1D9C2DAC3DBC4EDD6B9FD79EEB90C
:1039E400E579B9FE79F5B9D179B9E379B9E279B96B
:1039F400D279B9F179B9EA79B9D379B9EB79B9CC92
:103A040079B9D479B9EC79B9D579B9E479B9FC79CA
:103A1400B9F479B9CD79B9F779B9CA79B9E979B984
:103A2400F279B9F379B9FB79B9C979B9FA79B9CB2A
:103A340079B9E179B9ED79C6B9D679F6CFB9CE7944
:103A4400D1E3E2D2F1EAD3EBCCD4ECD5E4FCF4CD6F
:103A5400F7CAE9F2F3FBC9FACBE1B9C579AFDD6F77
:103A6400B9E379AFF66FAFCE6FAFC76FE0E8F0D8C8
:103A7400B9E079B9E879B9F079B9D879B9C8799759
:103A8400C757B9F87997DC57B9DE79C0AFDF6FAFA4
:103A9400C16FAFD96FAFC26FAFDA6FAFC36FAFDBB8
:103AA4006F97C257B9D07997DB5797D957E7AFECDF
:103AB4006FAFCC6FAFF26FAFF56FAFD36FAFC56FB2
:103AC400AFE46FAFC66FB9C679AFD56FAFF76FAF5D
:103AD400D26FAFE16FAFE96FAFCD6FAFD16FAFF121
:103AE4006FAFCA6FAFC96FAFEB6FAFD46FAFD56FA6
:103AF400AFCB6FAFF36FAFF46FB9F579AFEA6FAFD8
:103B0400E26FAFFA6FAFE26FAFE36FB9CE79D1E393
:103B1400E2D2F1EAD3EBCCD4ECD5E4FCF4CDF7CA91
:103B2400E9F2F3FBC9FACBE1B9C579AFDD6FB9E3CB
:103B340079AFF66FAFCE6FE7AFEC6FAFCC6FAFF28C
:103B44006FAFF56FAFD36FAFC56FAFE46FAFC66F35
:103B5400B9C679AFD56FAFF76FAFD26FAFE16FAFC3
:103B6400E96FAFCD6FAFD16FAFF16FAFCA6FAFC9B0
:103B74006FAFEB6FAFD46FAFD56FAFCB6FAFF36FEA
:103B8400AFF46FB9F579AFEA6FAFE26FAFFA6FAF29
:103B9400E26FAFF66F0000000000000000000000BC
:103BA4000000000000000000000000000000000011
:103BB4000000000000000000000000000000000001
:103BC40000000000000000000000000000000000F1
:0E3BD40000000000005AFF2000730A000000ED
:020000021000EC
:10E000007EC00000BFC00000A3C00000A1C000008F
:10E010009FC000009DC000009BC0000099C0000090
:10E0200097C0000095C0000093C0000091C00000A0
:10E030008FC000008DC000008BC0000089C00000B0
:10E0400087C0000085C0000083C0000081C00000C0
:10E050007FC000007DC000007BC0000079C00000D0
:10E0600077C0000075C0000073C0000071C00000E0
:10E070006FC000006DC000006BC0000069C00000F0
:10E0800067C0000065C0000063C00000BBBEEC2D8F
:10E09000FD2DB7B6B0FCFDCF27BFE895B7B6B0FCF5
:10E0A000FDCF21E1B7B6B6FCF4CF0895040309040F
:10E0B0001C037700770077002E006600690073006C
:10E0C000630068006C002E00640065000E035500BC
:10E0D0005300420061007300700012011001FF0044
:10E0E0000008C016DC05020101020001090212004D
:10E0F000010100803209040000000000000011242A
:10E100001FBECFEFD0E4DEBFCDBF34B7D0E4CEEF3B
:10E110002991203F299109F02FEF20933F0130935F
:10E12000400111E0A0E0B1E0E2EAF9EE01E00BBF4E
:10E1300002C007900D92A630B107D9F711E0A6E012
:10E14000B1E001C01D92AF33B107E1F79FD127C401
:10E1500057CFA82FB92F80E090E041E050EA6095BA
:10E1600030E009C02D9182279795879510F084277C
:10E170009527305EC8F36F5FA8F30895EADF8D93AB
:10E180009D930895CF93CFB7CF93DF93C395499BCA
:10E19000E9F7499B0BC0499B09C0499B07C0499BB4
:10E1A00005C0499B03C0499B01C089C06F93C091C2
:10E1B0002201DD27C75DDE4F2F9365E5499B03C034
:10E1C0002F916F91E6CF0F931F934F9320E040E183
:10E1D0005F9309B1067001FB27F93F9350E03BE0E4
:10E1E00039C0167040642F77012F5F5F1EC04068F2
:10E1F00019B116702F7752501FC0406409B12F77A4
:10E200000670D1F15F5F00C023C0406219B12F7763
:10E21000167091F15F5F00C025C006701027515045
:10E2200012F45D5F0000115027952C3F19B1C8F61C
:10E2300016700127015027952C3FC8F642274993B5
:10E2400009B1067010274F73115027952C3FA8F67F
:10E250004695469519B1167079F00127015027951A
:10E260002C3F98F66B5A60F3315009B1B0F600C0FC
:10E2700011E01CBB002717C03B503195C31BD04099
:10E2800011E01CBB0881033CF9F00B34E9F020914C
:10E2900020011981110F1213EDCF093651F10D3202
:10E2A00011F0013E39F7009327013F915F914F91A3
:10E2B0001F910F912F916F91CCB3C0FD67CFDF916C
:10E2C000CF91CFBFCF91189520912701222369F3D9
:10E2D00010912501112339F534303AF1309325019D
:10E2E00020932101109122013BE0311B3093220148
:10E2F0001CC0009125010130B4F40AE53091000101
:10E3000034FD14C000930001C5E1D1E013C005271E
:10E3100010E000C000000BB91AC0052710E0221F52
:10E320001DC010E021C04AE502C032ED432FC4E118
:10E33000D0E032E01AB11660599A0BB11AB956E022
:10E3400020E865E320FF05270BB9279517951C3FAB
:10E35000F0F66695B8F7B1F720FF05270BB92795BA
:10E3600017951C3FD0F62795179517FF0527000036
:10E370001C3F0BB9B0F629913A9519F7097F109116
:10E380002601110FC651D0400BB911F01093200196
:10E3900011E01CBB02601AB1197F402F497F54E085
:10E3A0005A95F1F70BB91AB94BB97FCFFB01A89574
:10E3B00031978040E1F70895DC0113963C91139763
:10E3C0001496EC91149712962C911297203331F4F5
:10E3D000E370F0E0EE5FFE4F80810895932F8E2F63
:10E3E000283549F4332391F4E1E0F0E089E08093AB
:10E3F0005700849108952035E1F4332389F4E0E057
:10E40000F0E089E08093570084910895383009F056
:10E4100036C0E3E0F0E089E08093570084910895EE
:10E42000383069F5E2E0F0E089E0809357008491AC
:10E430000895203251F4A0E0B0E0880F991FAA1F80
:10E44000BB1FABBFFC0187910895283269F4A0E09F
:10E45000B0E0880F991FAA1FBB1F0196A11DB11D17
:10E46000ABBFFC0187910895203A09F46AC2203CB1
:10E4700021F415966C9172D202C02F3F11F080E00A
:10E48000089581EF80930B0180E008951AB881E030
:10E490008BB985BF82E085BF60E071E787DF04B696
:10E4A00003FE0EC08EEF9FE054D210E0805B904BD5
:10E4B00009F411E08EEF9FE06FEF7FEF5DD208C0AF
:10E4C00004B601FC02C010E003C019B11095117030
:10E4D00014BE112309F427C28EEF80930B0114BEE2
:10E4E00088E10FB6F89480936000109260000FBE30
:10E4F00080916900826080936900E89A519A8CE06B
:10E5000060E075E353DF5198789481EF80930B01BD
:10E5100090912501935097FD52C180912201CCE04A
:10E52000D0E0C81BD109C75DDE4F809121018D323B
:10E5300009F0C2C0983009F040C183EC8093150106
:10E540008AE58093000110920A013881832F80763A
:10E550002981882309F441C086E091E09093240149
:10E5600080932301233031F4CE0126DF809309010B
:10E5700024E098C0253079F12A3069F1822F845047
:10E580008630E0F48A819B8190930D0180930C0189
:10E59000293039F48C819D8190930F0180930E0175
:10E5A00018C08E81809310018D818270809311013B
:10E5B0002093120137FD71C09FEF70C0223021F40B
:10E5C00080910B018E7F03C080910B01816080934D
:10E5D0000B0120E067C021E065C08A8110921E0116
:10E5E000222331F410921F018EE191E022E050C00D
:10E5F000253019F48093260148C02630B1F58B816F
:10E60000813019F48AED90EE04C0823041F48CEE32
:10E6100090EE909324018093230122E122C0833065
:10E62000F9F48A81882341F48CEA90EE90932401D6
:10E630008093230124E015C0813041F480EB90EEFB
:10E6400090932401809323012CE10BC0823041F48C
:10E650008CEC90EE90932401809323012EE001C076
:10E6600020E080E480930A011DC0283019F488E27C
:10E6700091E009C0293019F48093280106C02A309E
:10E6800021F48EE191E021E003C08EE191E020E0F1
:10E69000909324018093230105C09E8180E880939C
:10E6A0000A0107C08F81882319F49E81921708F010
:10E6B000922F9093010181C080910A0187FF7DC054
:10E6C00080911001092F891708F4082F801B80936F
:10E6D0001001FF24882311F4FF24F39410E066C096
:10E6E00080911201873070F080910C0190910D01A2
:10E6F000019690930D0180930C01019769912ED1A1
:10E700001F5F54C040910C0150910D0160910E01AA
:10E7100070910F01403080EE580781E0680780E07B
:10E72000780708F048C01E5FF8948991999121E01C
:10E730000C01FA0160935B0020935700E8951124C7
:10E740007894DB01CA010296A11DB11D80930C01D2
:10E7500090930D01A0930E01B0930F01882341F017
:10E76000FF2021F1101710F1809111018823F1F0A1
:10E77000F89483E0FA0160935B0080935700E8957A
:10E78000789407B600FCFDCFF89485E0FA01609319
:10E790005B0080935700E895789407B600FCFDCFA6
:10E7A000F89481E180935700E8957894101708F465
:10E7B00097CFFF2011F01092010110922501809156
:10E7C000000184FF8CC0809101018F3F09F487C054
:10E7D000182F893008F018E0811B80930101809187
:10E7E000150198E8892780931501112309F465C064
:10E7F00080910A0187FF3DC080911001811708F4C4
:10E80000182F811B8093100100911201C6E1D1E005
:10E8100028C0073030F080910C0190910D0191D00B
:10E820000BC080910C0190910D01A0910E01B0914F
:10E830000F01ABBFFC0187918883219680910C0169
:10E8400090910D01A0910E01B0910F010196A11DB3
:10E85000B11D80930C0190930D01A0930E01B09314
:10E860000F01812F90E08A5E9E4FC817D90789F665
:10E8700022C0C0912301D091240186FF11C0212F15
:10E8800046E151E0CE01A0E0B0E0A160ABBFFC01E9
:10E890008791FA018193AF012196215099F707C022
:10E8A000912FE6E1F1E0899181939150E1F7D093C6
:10E8B0002401C0932301193060F486E191E0612FB7
:10E8C0005DDC612F6C5F6C3041F08FEF8093010154
:10E8D00004C08FEF809301016EE16093000194E129
:10E8E00089B1867031F49150D9F7109226011092B7
:10E8F000200180910B01803130F0489B0FC0809146
:10E900000B01805109C0489909C080910B018230E8
:10E9100028F080910B01825080930B0180910B01B4
:10E92000882309F0F5CDF894519A1BB81DBA1092BE
:10E93000690081E085BF15BEE0911301F0911401DB
:10E940000995F999FECF92BD81BDF89A992780B5B6
:10E950000895A8E1B0E042E050E013C0262FF999F5
:10E96000FECF1FBA92BD81BD20BD0FB6F894FA9AB2
:10E97000F99A0FBE01960895F1DF272FF0CFDC0141
:10E98000CB01FC01F999FECF06C0F2BDE1BDF89ABA
:10E99000319600B40D9241505040B8F70895F89464
:02E9A000FFCFA7
:06E9A2005AFF1E9705005C
:040000031000E00009
:00000001FF
